:1000000018C1000032C1000030C100002EC1000044
:100010002CC100002AC100000C9406090C9415099B
:1000200024C1000022C1000020C100001EC1000048
:100030001CC100001AC1000018C1000016C1000058
:1000400014C1000012C1000010C100000EC1000068
:100050000CC100000AC1000008C1000006C1000078
:100060000C94F1090C94FC0900C10000FEC00000D2
:10007000FCC00000FAC00000F8C00000F6C000009C
:10008000F4C00000F2C00000F0C00000EEC00000AC
:10009000ECC00000EAC00000E8C00000E6C00000BC
:1000A000E4C00000E2C00000E0C00000DEC00000CC
:1000B000DCC00000DAC00000D8C00000D6C00000DC
:1000C000D4C00000D2C00000D0C00000CEC00000EC
:1000D000CCC00000CAC00000C8C00000C6C00000FC
:1000E000C4C00000C2C00000C0C00000BEC000000C
:1000F000BCC00000BAC00000B8C00000B6C000001C
:10010000B4C00000B2C00000B0C00000AEC000002B
:10011000ACC00000AAC00000A8C00000A1C400003C
:10012000A4C00000A2C00000A0C000009EC000004B
:100130009CC000009AC0000098C0000096C000005B
:1001400094C0000092C0000090C000000C946609AA
:100150008CC000008AC0000088C0000086C000007B
:1001600084C0000082C0000080C000007EC000008B
:100170007CC000007AC0000078C0000076C000009B
:1001800074C0000072C0000070C000006EC00000AB
:100190006CC000006AC0000068C0000066C00000BB
:1001A00064C0000062C0000060C000005EC00000CB
:1001B0005CC000005AC0000058C0000056C00000DB
:1001C00054C0000052C0000050C000004EC00000EB
:1001D0004CC000004AC0000048C0000046C00000FB
:1001E00044C0000042C0000040C000003EC000000B
:1001F0003CC000000C94DF130C9497140D040F0402
:10020000110413041504170419041B04C80BEE0B86
:10021000150C3E0C470C4C0C910C960CB50CBC0C00
:10022000C40C580C600C680C730C750C770C7F0CAC
:10023000870C11241FBECFEFCDBFDFE2DEBF10E27F
:10024000A0E0B0E2E0E5FBE202C005900D92AA3B1F
:10025000B107D9F72DE2AAEBB0E201C01D92AC3F85
:10026000B207E1F791D20C94A615CACE84E0809330
:1002700056008CE1BDD3809363008BEB80936600C6
:1002800080E88093650081E08093600088ED84BF02
:100290001092410083E080935000809151008330A0
:1002A000E1F78091500081608093500088E1809355
:1002B00055008091510080FFFCCF809150008061FB
:1002C000809350008091510084FFFCCF88ED84BF63
:1002D00084E0809340000895E0E7F0E085818E7F20
:1002E0008583E0E0FAE08FEB9DE586A397A380EE9F
:1002F0009EE280A391A382E0808308958091200AEA
:100300009091210A813E2EE2920718F020919E23BF
:1003100006C0803E2EE2920721F020919B2320937D
:100320006A0020910520222321F080910520815030
:1003300033C0885F9A42813D974080F11092BA2085
:100340008091BB209091BC20A091BD20B091BE2097
:100350000196A11DB11D8093BB209093BC20A0935A
:10036000BD20B093BE208091BB209091BC20A09175
:10037000BD20B091BE20892F9A2FAB2FBB27809331
:10038000BE238091BB209091BC20A091BD20B09154
:10039000BE208093BD2386E08093052080910720B6
:1003A000909108200196B1F4809109208F3F91F03F
:1003B00080910620811106C0809106208150809393
:1003C00006200895809114019091150180930720D3
:1003D000909308200895009709F45EC00CF457C06C
:1003E00040E020916B0030E020939C2330939D23CC
:1003F00020919C2330919D233695322F22273795CB
:10040000279520939C2330939D2350916A0020913F
:100410009C2330919D23250F311D20939C233093E5
:100420009D23000020919C2330919D23281739079C
:1004300028F410929C2310929D23089520919C23D0
:1004400030919D23280F391F2115304238F08FEF4E
:100450009FE180939C2390939D23089520919C235A
:1004600030919D23442329F0A901481B590BCA014F
:1004700002C0820F931F80939C2390939D238091B1
:100480009C2390919D238F7780936A000895919586
:100490008195910941E0A5CF0895CF93DF93C09155
:1004A000200AD091210A80910320909104209E017E
:1004B000281B390B20939F233093A0238091BA20CF
:1004C00081114BC080919F239091A0238E3C9F4F20
:1004D000D4F480919F239091A0238B369F4F9CF062
:1004E00080910220882321F080910220815008C051
:1004F00080916A0080939E2381E08093BA208CE0F3
:10050000809302202AC08CE08093022080919F2358
:100510009091A0238A369F4F1CF08FEF9FEF02C06F
:1005200081E090E08093992390939A2380919F2378
:100530009091A0232091992330919A2360E370E059
:100540000E947D15261B370B2093992330939A2305
:100550008091992390919A233EDF8091BA20813037
:1005600029F580919F239091A023C39794F08091C7
:100570000220882331F08091022081508093022054
:1005800015C080916A0080939B2383E08093BA20FA
:100590000DC080919F239091A023873991051CF471
:1005A00081E090E002C08FEF9FEF15DFC093032042
:1005B000D0930420DF91CF9108958617970779F0A3
:1005C0006817790728F49C01261B370BB90109C06D
:1005D0008617970718F4681B790B03C0089560E02D
:1005E00070E0CB010895CF93DF938091002090912C
:1005F0000120892B51F080910020909101200197DA
:10060000809300209093012043C080E490E0809389
:10061000002090930120809107209091082001965E
:10062000B9F1809114019091150120910920263093
:1006300018F467E771E002C06EEE72E00E9469157F
:10064000EC0180910720909108208C179D0758F4A9
:100650006091072070910820CE01AFDF029718F05B
:1006600080EC9DE511C08091072090910820C8176B
:10067000D90770F46091072070910820CE019DDFAA
:10068000029730F08FEB9DE58093360A9093370AFE
:10069000DF91CF910895AC01460F571F861B970B32
:1006A0002091200A3091210A24173507C8F720919C
:1006B000200A3091210A8217930790F70895E0E805
:1006C000F6E08FE0808385E0848308951F93CF93C5
:1006D000DF93C0E4D0E0198180E4898340E250E0F8
:1006E00064ED7DE280E290E00E942B0F1983DF91A0
:1006F000CF911F9108951F93CF93DF93C0E4D0E073
:10070000198180E4898387ED97E20E94610F81E07F
:100710000E94730F1983DF91CF911F91089508955F
:100720000F931F93842F50E0415851099DE7949FE8
:100730009001959F300D112490910920953048F437
:10074000843810F029583E4F9091C42067E771E03B
:1007500004C09091C4206EEE72E0969FA001979F16
:10076000500D1124420F531F4850584D00E913E01B
:100770002DE730E060E00E941C131F910F91089557
:100780001CBEEEEFF0E40994A1DF8091D42D882304
:1007900069F080E2E4EDFDE2A7EDB7E201900D9291
:1007A0008A95E1F71092D727A6DFEADF87E08093EA
:1007B000A20078945BDDB3DF7AD765D188D160E0A1
:1007C00080E01FD10BD18CE0FFD03ED5E2D5FBD528
:1007D00076DF60EA70E28AEA93E20E949F150000E9
:1007E0000000000000000000000000000000000009
:1007F000000000000000000000008091BF2088235E
:1008000071F3E091D6258E2F90E088309105A0F409
:10081000FC01E250FF4F0C94901584D10DC0F2D131
:100820000BC077D209C0F9D207C083D305C00AD460
:1008300003C009D401C078D41092BF20D0CF08954E
:100840000895809114018093B323809115018093C2
:10085000B423809124018093B52380912501809356
:10086000B6238091200A8093BF238091210A809330
:10087000C02380911401909115018634914080F03D
:100880008091140190911501893A914048F480912A
:100890001401909115018093F42D9093F52D000093
:1008A0008091C220882339F017DD1092C22081E0A8
:1008B0008093C12008958091C120882341F08091C8
:1008C000BA20833019F41ADD8EDE01C0E6DD809196
:1008D000C020882351F080911401909115018093DC
:1008E000F42D9093F52D1092C02080910920209135
:1008F000140130911501853028F481E0273731400B
:1009000030F004C081E02E3E324008F080E0809359
:10091000C42008950F931F9381E08093C720809394
:10092000C22000E913E02DE730E048EF57E260E035
:1009300081E80E941C132DE730E045E758E260E0B3
:1009400082E80E941C132DE730E042EF58E260E09D
:1009500083E80E941C132DE730E04FE659E260E087
:1009600084E80E941C132DE730E04CEE59E260E071
:1009700085E80E941C132DE730E049E65AE260E06A
:1009800086E80E941C1381E01F910F910895109238
:10099000C720089581E0089581E008951092200213
:1009A000982F9C7193689093200287FF03C080E189
:1009B00092E002C080E090E0892B809321021092A7
:1009C0002202109226020895E0E0F2E010AA836865
:1009D00080AB80E181AB12AA16AA0895E0E0F2E0B4
:1009E00010A683E880A78FE281A712A616A6089515
:1009F000AAECB1E092E09C93E82FF0E084911C9285
:100A00000895909171009D7F909371001092000263
:100A1000623011F09CE101C09EE19093010290E4EC
:100A200090930202811102C080E401C080EC8093A7
:100A30000302613011F084E001C083E0809304027E
:100A400080E2D6DF80930C0281E2D2DF80930D0238
:100A5000109218021092190281E080930002BECF1A
:100A60001F920F920FB60F9211248F930000000077
:100A70000000000081E0809323028F910F900FBE51
:100A80000F901F901895CF93DF93E0E7F0E08281FD
:100A90008B7F8283C0E2D3E08DE0888380E489830A
:100AA00089E08A8383E3A4DF888782E3A1DF8987E3
:100AB00087E39EDF8A8786E39BDF8B87E0E2F6E0B1
:100AC0008081836080831482DF91CF910895E0E775
:100AD000F0E080818E7F808383E880930001089519
:100AE000E0E0F1E0108A80E4808B10A280A310AADD
:100AF00080ABE0E4F1E0108280831092C620109277
:100B0000C5201092C4201092A8231092A9231092FD
:100B1000A6231092A72308958093D62581E0809381
:100B2000BF200895CF93DF9310920920D9DFC0E052
:100B3000D1E01EAA84E288AB19AA49E54AAB32E0AB
:100B40003BAB60910B2070910C206CAB7DAB67EDE3
:100B500075E268AF79AF1AAE9BE39CAF93E09DAFAF
:100B60001EAE28A9206828AB10924601E0E4F1E00F
:100B70008083109241014093420190934301409140
:100B80000D2050910E20409344015093450146ECB6
:100B900053E2409348015093490110924A0129E3DE
:100BA00020934C0190934D0110924E0190819068DA
:100BB0009083188A90E4988B888B198A95E99A8B90
:100BC00090E19B8B4EEE52E04C8B5D8B888F398F82
:100BD0001A8E88EF97E28C8F9D8F1E8E68EC70E0E6
:100BE00084EF91E058DD88EC90E0809307209093AB
:100BF000082081E08093062088898068888BDF91B7
:100C0000CF9108951F93CF93DF9311E010930920A4
:100C100067DFC0E0D1E018AA80E488AB84E088AB4D
:100C200019AA1AAA4BE44BAB1CAA1DAA1EAA8AE059
:100C300090E288AF99AF1AAE60EA6CAF38E03DAF92
:100C40001EAE88A9806A88ABE0EAF8E085E580837B
:100C5000808310924601E0E4F1E084E28083109208
:100C6000410199E59093420122E020934301A09134
:100C70000B20B0910C20A0934401B0934501A7ED47
:100C8000B5E2A0934801B093490110924A019BE359
:100C900090934C0193E090934D0110924E019081FE
:100CA0009068908388A319A295E99AA34BA34EEE6E
:100CB00052E04CA35DA368A739A71AA666EE7AE2B4
:100CC0006CA77DA71EA6888B198A9A8B90E19B8BB7
:100CD0004C8B5D8B888F298F1A8E88EF97E28C8FD3
:100CE0009D8F1E8E68EC70E084EF91E0D4DC88EC80
:100CF00090E080930720909308201093062088A10D
:100D0000806888A388898068888BDF91CF911F9144
:100D100008951F93CF93DF9312E010930920E0DE34
:100D2000C0E0D1E01EAA84E288AB19AA39E53AAB4B
:100D30001BAB40910B2050910C204CAB5DAB47EDB1
:100D400055E248AF59AF1AAE9BE39CAF93E09DAF1D
:100D50001EAE28A9206828AB10924601E0E4F1E01D
:100D6000808310924101309342019093430120917E
:100D70000D2030910E20209344013093450126EC44
:100D800033E2209348013093490110924A0129E34C
:100D900020934C0190934D0110924E0190819068E8
:100DA0009083188A90E4988B888B198A45E94A8B3E
:100DB00090E19B8B2EEE32E02C8B3D8B888F198F30
:100DC0001A8E68EF77E26C8F7D8F1E8E88A319A232
:100DD0004AA39BA32CA33DA384E388A719A71AA623
:100DE00086EE9AE28CA79DA71EA668EC70E084EFC1
:100DF00091E051DC88EC90E08093072090930820EC
:100E000081E08093062088898068888B88A180682B
:100E100088A3DF91CF911F9108951F93CF93DF9304
:100E200013E0109309205CDEC0E0D1E0109246018F
:100E3000E0E4F1E084E280831092410129E520930F
:100E4000420192E09093430140910B2050910C207D
:100E5000409344015093450147ED55E240934801CA
:100E60005093490110924A019BE390934C011093D7
:100E70004D0110924E019081906890831EAA88AB1C
:100E800019AA2AAB1BAB20910D2030910E202CAB60
:100E90003DAB26EC33E228AF39AF1AAE99E39CAFF5
:100EA0001DAF1EAE98A9906898AB18A250E458A345
:100EB00094E098A319A21AA24BE44BA31CA21DA272
:100EC0001EA22AE030E228A739A71AA630EA3CA7DA
:100ED00028E02DA71EA698A1906A98A395E5909367
:100EE000A008188A588B888B198A85E98A8B4B8BC6
:100EF0008EEE92E08C8B9D8B388F298F1A8E88EF27
:100F000097E28C8F9D8F1E8E68EC70E084EF91E0ED
:100F1000C2DB88EC90E0809307209093082081E06A
:100F20008093062088898068888BDF91CF911F91FC
:100F300008951F93CF93DF9314E010930920D0DD21
:100F4000C0E0D1E018AA80E488AB18AB19AA1AAAAD
:100F50003BE43BAB1CAA1DAA1EAA8AE090E288AF24
:100F600099AF1AAE50EA5CAF88E08DAF1EAE98A97B
:100F7000906A98AB95E59093A00810924601E0E442
:100F8000F1E094E290831092410129E5209342011F
:100F900022E02093430160910B2070910C2060931C
:100FA00044017093450167ED75E2609348017093C9
:100FB000490110924A012BE320934C0123E0209336
:100FC0004D0110924E01208120682083988B198A50
:100FD00045E94A8B3B8B2EEE32E02C8B3D8B588FB4
:100FE000898F1A8E68EF77E26C8F7D8F1E8E98A3A3
:100FF00019A24AA39AE49BA32CA33DA393EC98A720
:1010000089A71AA686EE9AE28CA79DA71EA668EC71
:1010100070E084EF91E03FDB88EC90E08093072064
:101020009093082081E08093062088898068888BCF
:1010300088A1806888A388898061888BDF91CF919F
:101040001F910895FFCFCF93DF9386E0809309200F
:1010500047DDC0E0D1E01EAA84E288AB19AA39E5D9
:101060003AAB93E09BAB40910D2050910E204CABDE
:101070005DAB46EC53E248AF59AF1AAE29E32CAF53
:101080009DAF1EAE28A9206828AB10924601E0E46F
:10109000F1E08083109241013093420122E02093DD
:1010A000430140910B2050910C20409344015093F8
:1010B000450147ED55E24093480150934901109294
:1010C0004A013BE330934C0190934D0110924E0145
:1010D000908190689083188A90E4988B888B198A05
:1010E00095E99A8B90E19B8B4CED55E04C8B5D8B99
:1010F000888F298F1A8E88EF97E28C8F9D8F1E8E96
:1011000068EC70E084EF91E0C6DA80E991E08093CA
:1011100007209093082081E08093062088898068CA
:10112000888BDF91CF910895CF93DF9387E08093F1
:101130000920D6DCC0E0D1E01EAA84E288AB19AA5F
:1011400039E53AAB93E09BAB40910D2050910E20D6
:101150004CAB5DAB46EC53E248AF59AF1AAE29E356
:101160002CAF9DAF1EAE28A9206828AB1092460177
:10117000E0E4F1E08083109241013093420122E0EB
:101180002093430140910B2050910C204093440147
:101190005093450147ED55E2409348015093490172
:1011A00010924A013BE330934C0190934D01109211
:1011B0004E01908190689083188A90E4988B95E214
:1011C000988B198A95E99A8B90E19B8B4CED55E0B1
:1011D0004C8B5D8B888F298F1A8E88EF97E28C8FCE
:1011E0009D8F1E8E68EC70E084EF91E054DA80E908
:1011F00091E0809307209093082081E0809306205F
:1012000088898068888BDF91CF9108951F920F9213
:101210000FB60F9211248F9381E0809303018F9179
:101220000F900FBE0F901F9018951F920F920FB640
:101230000F9211248F9382E0809303018F910F907E
:101240000FBE0F901F901895E0E7F0E083818C7F30
:10125000838384818C7F848380818D7F8083E0E899
:10126000F1E080EC8283128688EC81831186A0E015
:10127000B8E034E03C9323E011962C931197149638
:101280001C92149785ED91E096968D939C93979779
:1012900016961C921697E0E4F8E0308321831482BE
:1012A00086A397A31682E0E6F6E0808180618083C2
:1012B000E0E4F9E083E18183148282E08683A6A3DF
:1012C000B7A310A611A681E0808308951F920F9204
:1012D0000FB60F9211242F933F934F935F938F93E9
:1012E0009F93CF93DF931F92CDB7DEB78FEF80939D
:1012F0004C0980910920873031F480912C02898338
:1013000090912D0202C090912C028091C320891BE4
:10131000209168093091690982308CF02A3F37406A
:1013200070F4209168093091690989301CF481E0DA
:1013300090E002C086E090E0820F931F18C02091D9
:101340006809309169098F3FB4F42730310598F06E
:101350002091680930916909883F1CF081E090E094
:1013600002C086E090E0A901481B590BCA01809396
:101370007809909379090F90DF91CF919F918F9188
:101380005F914F913F912F910F900FBE0F901F9043
:101390001895E0E7F0E083818F7E8383E0E4F6E058
:1013A00080818A6A80838FEF848388E5828BE0EA7C
:1013B000F8E080E3838384EC858387E0868317826B
:1013C00088E184830895E0E7F0E08381877F838369
:1013D000E0ECF8E0118288E58093550680E6808392
:1013E00008951F920F920FB60F92112400000F90D4
:1013F0000FBE0F901F9018951F920F920FB60F926D
:1014000011248F93EF93FF93E0EAF8E080818083CB
:10141000FF91EF918F910F900FBE0F901F90189535
:101420009FB7F894A0E5B0E016968C911697897F47
:1014300016968C931697E0E6F0E080E885838BEBB8
:10144000868316968C911697846016968C9380816D
:10145000816080839FBF08959FB7F894E82FF0E0E4
:10146000E059FF4F60958081682360839FBF089596
:10147000CF93863011F0C0E001C0C8E180915100E7
:1014800081FD0DC09FB7F8948091500082608093D9
:1014900050009FBF8091510081FFFCCFC1DF6C2FB6
:1014A000636084E490E0BCD460E480E0CF91D4CF6A
:1014B0008091C82008958091C820813009F467CABE
:1014C0000895F0D0FC0183818093C820811101C070
:1014D00021CA81E008959091C625892F807697FFD3
:1014E00007C0803491F48091C72581110EC054CA81
:1014F000803459F48091C725811107C08091CC2593
:101500009091CD25892B09F045CA80E008958091FE
:10151000C8258F770C94A6129091D020911102C00B
:1015200080E00895E091CD20F091CE200190F081EF
:10153000E02D94818917A0F7E093CB20F093CC2085
:10154000228133812E0F3F1FE217F30798F4918118
:10155000943061F49281891309C09381691306C0A4
:10156000E093CB20F093CC2081E008959081E90FA7
:10157000F11DEACFE093CB20F093CC20D1CFE091C6
:10158000CD20F091CE200190F081E02D2281338199
:101590002E0F3F1FFC014081E40FF11DE217F307FE
:1015A00048F48181843031F0853039F08081E80F52
:1015B000F11DF4CF80E090E00895CF0108951F93CE
:1015C000CF93DF93182FA8DF882339F1C091CB2068
:1015D000D091CC20CE01D3DFEC01892B41F04C819E
:1015E0005D816B818A81BFD78111F4CF16C0E091F4
:1015F000CD20F091CE2092818381E92FF82FE10F49
:10160000F11DE10FF11D0190F081E02D0190F081BD
:10161000E02DDF91CF911F91099480E0DF91CF9170
:101620001F910895EF92FF921F93CF93DF93C82FDE
:1016300060E072DF811102C010E02DC0E091CD208A
:10164000F091CE2092818381E92FF82FEC0FF11DCC
:10165000EC0FF11DE080F180D7011696ED91FC9121
:1016600017970995682F8C2F57DF182F882321F3A0
:10167000C091CB20D091CC20CE0181DFEC01892B11
:1016800021F08A810E94C613F7CFD7011296ED91FF
:10169000FC9113970995812FDF91CF911F91FF90B6
:1016A000EF9008958091CB209091CC200895E2C6D0
:1016B000CF938091D020882311F0C0E008C0109211
:1016C000D0201092D4201092D520CF910895E0918F
:1016D000CD20F091CE200190F081E02D8481C817BB
:1016E00070F78C2F9FDFCF5FF2CFCF938091D02008
:1016F0008823F1F0C0E0E091CD20F091CE20A081D0
:10170000B18114968C91C81798F492818381E92F46
:10171000F82FEC0FF11DEC0FF11D0190F081E02D81
:101720000084F185E02D309709F00995CF5FE3CF74
:10173000CF9108950F931F93CF93DF931092D025ED
:101740001092D1251092D2251092D3251092D42533
:101750001092D5258091C62587FF07C02091CC2502
:101760003091CD25232B09F455C38076803409F0C0
:101770000FC1E091C7258E2F90E0FC01E05AF109DE
:10178000EB30F10508F004C1EA5FFE4F0C949015B0
:1017900081E08093C0208091072090910820809361
:1017A000B72380910720909108209093B8238091CF
:1017B0009E238093B92380919B238093BA238091A9
:1017C0006A008093BB2380916B008093BC2360915F
:1017D000CC257091CD258AEA93E2D4C010920008FE
:1017E0008091C8259091C925809336089093370839
:1017F0008091CA258F70809300086091CC257091EC
:10180000CD2586EC93E2A8D68091CC259091CD256C
:1018100020910D2030910E208217930709F4C5C244
:1018200080930D2090930E2026C010924008809146
:10183000C8259091C9258093760890937708809168
:10184000CA258F70809340086091CC257091CD257A
:1018500087ED95E281D68091CC259091CD25209180
:101860000B2030910C208217930709F49EC28093BD
:101870000B2090930C208091092051C01092680990
:10188000109269098091C8258093C3208EC28091EF
:10189000C8258093240689C2E091C825F091C92506
:1018A000E830F10508F074C0EF5EFE4F0C9490151F
:1018B00060E080E0A6D88091CA2570D880E02FC073
:1018C00060E080E09ED88091CA2568D881E027C07A
:1018D00061E081E096D88091CA2560D88091CB25BF
:1018E00073D882E01CC083E01AC084E018C060E0B6
:1018F00080E087D88091CA2551D885E010C061E08A
:1019000080E07FD88091CA2549D886E008C062E08F
:1019100080E077D88091CA25806840D887E0FCD8DD
:1019200044C28091C825809384063FC28091C82517
:101930009091C925892B91F00E94660380E2E4ED25
:10194000FDE2A7EDB7E201900D928A95E1F781E003
:101950008093D7270E947B030E946603E9E7F0E0AB
:1019600091E088EDF89484BF90836091CC257091CC
:10197000CD258AEA90E206C06091CC257091CD25F4
:1019800089EA90E2E9D511C20E948A0481110DC250
:101990008091C625982F907609F0C9C187FFFBC0BA
:1019A0002091CC253091CD252115310509F4BFC1F9
:1019B0008F7109F09EC08091C725863071F0883004
:1019C00009F48EC08111B3C12230310509F0AFC1D5
:1019D00062E070E084ED90E2D5CF8091C8259091CF
:1019E000C925292F332722303105A1F060F4213099
:1019F000310509F09CC18091192090911A20DC01D9
:101A00006C9170E05BC02330310589F12F303105D6
:101A100009F18DC1E0911920F0911A2021898217D6
:101A200008F085C19927880F991F880F991FE091A9
:101A30001B20F0911C20E80FF91F80819181FC018F
:101A40006281738189D5E091CE25F091CF2582E026
:101A5000818335C080911D2090911E20009709F44C
:101A600066C1DC0112966D917C91139727C099276E
:101A70008130910569F038F0029709F058C168E0AB
:101A80008AE890E208C064E070E08CE990E216C059
:101A900067E083E990E2282FAAE7B0E2FC01819198
:101AA00090E08D939D938E2F821B8617C0F3660F57
:101AB0006E5F6093782070E088E790E24DD580916A
:101AC000CC259091CD252091D0253091D12582171C
:101AD000930708F06AC18093D0259093D12565C102
:101AE0002130310509F023C161E070E080ED90E222
:101AF00049CF8130C1F58091C7258A3009F017C1DF
:101B00002130310509F013C18091D020882309F4D8
:101B10000EC1C091CA25D091CB250091CD20109146
:101B2000CE20D801ED91FC918481C81708F0FFC048
:101B300060E08C2FF1DC882309F4F9C0DD27CC0F9D
:101B4000DD1FF80182819381C80FD91FE881F981D7
:101B50000680F781E02D09958093D22061E070E046
:101B600082ED90E20FCF823009F0E1C08091C7256D
:101B70008111DDC02230310509F0D9C08091CA251C
:101B80003BD590E08093C9209093CA2062E070E03A
:101B900089EC90E2F7CE8F7109F07DC08091C72566
:101BA000833009F4C4C018F48130A1F0C0C085307E
:101BB00019F0893039F1BBC08091CC259091CD25A9
:101BC000892B09F0B4C087E89AE08093D2259093DE
:101BD000D325EBC08091CC259091CD25892B09F0A0
:101BE000A6C08091C8259091C925019709F09FC092
:101BF0008091D4209091D5208D7F8093D420909394
:101C0000D520D3C08091CC259091CD25892B09F08A
:101C10008EC09FD4882309F48AC02091C8253091B2
:101C2000C9253327E0911920F0911A20818990E08D
:101C30008217930708F47BC03BDD8091C825909103
:101C4000C9258093D020882309F4AFC099278150FB
:101C5000904C880F991F880F991F20911B2030915D
:101C60001C20820F931F8093CD209093CE20C0E044
:101C7000E091CD20F091CE200190F081E02D848183
:101C8000C81708F092C060E08C2F99DC882309F413
:101C90004EC0CF5FEDCF8130E9F48091C7258B3006
:101CA00009F045C08091CC259091CD25892B09F074
:101CB0003EC08091D020882309F439C0C091CA2544
:101CC000D091C8258C2FAEDC882389F16D2F8C2F05
:101CD00076DC2BC0823059F58091C725813019F010
:101CE000833089F024C08091CC259091CD25892B1B
:101CF000F1F48091C8259091C925892BC1F4809178
:101D0000CA2581D412C08091CC259091CD25892BF4
:101D100071F48091C8259091C925892B41F4809157
:101D2000CA2504D58091CA253AD581113EC080913B
:101D3000C6258F718130D9F58091D020882309F490
:101D400069C0C091CA25D091CB250091CD201091BA
:101D5000CE20D801ED91FC918481C81708F05AC0BB
:101D600060E08C2FD9DB882311F1FE01FF27EE0FF5
:101D7000FF1FD80112968D919C911397E80FF91FC0
:101D800000811181D8011696ED91FC911797099564
:101D9000682F8C2FC1DB882351F0D8011496ED9168
:101DA000FC9115970995882311F081E034C080914A
:101DB000C6258F71823071F58091D020882351F132
:101DC000C0E0E091CD20F091CE20A081B1811496A9
:101DD0008C91C817F8F492818381E92FF82FEC0FCA
:101DE000F11DEC0FF11D00811181D8011696ED91C6
:101DF000FC9117970995682F8C2F8EDB882351F063
:101E0000D8011496ED91FC91159709958111CDCFCC
:101E1000CF5FD7CF80E0DF91CF911F910F910895D1
:101E20001BBEFC0128ED24BF608308958091CF0183
:101E300087FDFCCF08951F93CF93DF93C0ECD1E0D3
:101E40001A858A8761E08BEC91E0EADF1A87DF91DF
:101E5000CF911F910895CF92DF92EF92FF920F934F
:101E60001F93CF93DF938C017B016A01DFDFCCEC02
:101E7000D1E0888188608883B801705FA601C701BE
:101E800055D68881877F8883DF91CF911F910F91ED
:101E9000FF90EF90DF90CF900895CF93DF93C82FFE
:101EA000D62FC4DFACECB1E08C9188608C93EC2F22
:101EB000F0E0F05FD0838C91877F8C93DF91CF919E
:101EC00008950F931F93CF938C01B0DFC0E0F8010A
:101ED00061918F018C2FE1DFCF5FC032C1F7CF91CD
:101EE0001F910F910895CF93C82FA0DF20E2C29FCA
:101EF000C0011124E0ECF1E012829183808385E33C
:101F0000CF9199CF4091CA01E62FF72F8093CA0154
:101F100084914093CA010895E82FF0E0EA50F24D11
:101F200080818F3F09F4FFCF9FB7F89480818F5F46
:101F300080839FBF0895E82FF0E0EA50F24D808142
:101F4000811101C0FFCF9FB7F894808181508083B9
:101F50009FBF0895CF93C82F80919823C11105C0CA
:101F6000882339F081E0E7DF04C0811102C081E0FD
:101F7000D3DFC0939823CF910895282F2F70082E78
:101F8000000C990B392F331F3327331F832F90E019
:101F9000820F911D820F911D23E0880F991F2A95B2
:101FA000E1F78C5D9C4D08950F93E8ECF4E080819F
:101FB0008F7D808380818F7D8083ECE2F3E202E07D
:101FC000059310922E2310922F2300E2069300E433
:101FD0000693E4E2F3E200E2069300E40693E6EC03
:101FE000F5E21486158616861786128613861092D9
:101FF00007230F9108950F9385E080930723EDE267
:10200000F3E204E00593E5E2F3E204E005930F91C7
:1020100008950F9383E08093072310922E2310924C
:102020002F23ECE2F3E202E006930F910895E09192
:10203000D225F091D325309709F009940895282FDF
:102040002F70082E000C990B392F331F3327331FA5
:10205000832F90E0820F911D820F911D029749E01E
:10206000489F9001499F300D1124C901895A9D4D07
:102070000895AF92BF92DF92EF92FF920F931F935A
:10208000CF93DF93D82EDBDFEC018D2D76DF7C0143
:10209000DC011196EC91E770E150E73040F4F0E09C
:1020A000EE0FFF1FE455FF4D0081118102C008E0D3
:1020B00010E02D813E818B819C814881D7FE4AC0F2
:1020C000F70166817781260F371F2D833E832817FE
:1020D0003907A1F1BC01621B730B9B01211574E050
:1020E000370738F02FEF33E0C901B801F2D4281BCD
:1020F000390B41FF0AC0C901B801EBD4AC0191E032
:10210000452B09F090E0892F01C080E0988180FB89
:1021100091F99883D70116961D921C9217971296E3
:102120002D933C93139729813A818D819E81820F53
:10213000931F14968D939C93159708C041FF78C008
:102140004D7F48831682178212821382F70102E0C4
:10215000069385C0D7011296AD90BC90139742FFAD
:102160000FC0E981FA81B801B4D4B0E4DB9EB001BC
:10217000112469567F4DAC01CF01820F931FD6D435
:102180002D813E812A0D3B1D2D833E838B819C81B9
:102190008217930710F48D839E83F7012681378180
:1021A000A216B30609F044C02D813E818217930721
:1021B00009F43EC0AC01421B530B9A01211554E0B7
:1021C000350750F02FEF33E0C901B80182D4B901CF
:1021D000681B790BCB0107C0C901B8017AD4D901BA
:1021E000A81BB90BCD01F70112821382801791074A
:1021F00098F4888184608883F0E4DF9EC001112414
:1022000089569F4DD70114968D939C9315971696DA
:102210000D931C9317979ACF49815A812D813E8146
:10222000240F351FF70124833583868397838ECF50
:10223000888180FF14C08E7F8883EF81F885309776
:1022400071F06D817E814D2D80E0DF91CF911F91E6
:102250000F91FF90EF90DF90BF90AF900994DF91C6
:10226000CF911F910F91FF90EF90DF90BF90AF90B3
:1022700008950F93CF93DF9380910723833029F440
:10228000D6DEDF91CF910F918FCE20910323309135
:102290000423C091D025D091D125C21BD30B61F569
:1022A0008091052390910623820F931F809305232D
:1022B000909306232091CC253091CD25821793074A
:1022C00021F08091D620882331F084E08093072389
:1022D000E4E2F3E236C0E091D425F091D5253097C1
:1022E00099F00995882381F010920323109204231A
:1022F000C091D025D091D125C034D10528F01092BD
:10230000D620C0E4D0E003C081E08093D620C09303
:102310002E23D0932F238091032390910423209187
:10232000CE253091CF25280F391F209330233093AD
:102330003123C80FD91FC0930323D0930423ECE2A9
:10234000F3E202E00693DF91CF910F9108950F938E
:10235000CF938091CC0480FF63C021E02093CC0414
:1023600084E293E2FC0100E80693ECE2F3E200E889
:1023700006932093CA04FC0100E106938091072391
:10238000882329F08350823008F451DE0DDE8091DD
:10239000262390912723089709F044C088E0E3ECB6
:1023A000F2E2A6ECB5E201900D928A95E1F78091F8
:1023B000C80480628093C8048091C80480628093BE
:1023C000C804B8D9C82F811102C015DE2BC0809176
:1023D000C62587FF0DC01092052310920623109288
:1023E00003231092042382E08093072342DF1BC063
:1023F0008091CC259091CD25892B11F40ADE13C054
:1024000010920523109206231092032310920423A6
:1024100081E080930723E4E2F3E202E0069303C045
:10242000C0E001C0C1E08C2FCF910F910895CF93F0
:10243000CFB7F89481E08EDDEAECF4E080E48083AD
:1024400080E28083E1ECF4E0808181608083A9EC0C
:10245000B4E08C9182608C93E8ECF4E0808180643D
:1024600080838C9181608C93808180688083CFBFD2
:10247000CF910895CF931092600080E30E94380AB4
:102480008091C00480648093C00481E080936000E8
:10249000CFB7F89480E090E0FC0123E0EE0FFF1F3F
:1024A0002A95E1F7E85FFC4D158E01968E30910577
:1024B00099F780E090E039E0389FF001399FF00D06
:1024C0001124E95AFD4D20812E7F208301968C3006
:1024D000910591F76AE170E082E014DD8F3F09F425
:1024E0008FE18093FA046BE170E082E00BDD8F3FB7
:1024F00009F48FE18093FB048091C004866080938F
:10250000C0048091C00480688093C0048091C0049E
:1025100080618093C00484E293E28093C604909328
:10252000C7048091C00480628093C0048FEF8093C1
:10253000C5048091C80482608093C80410929823D7
:1025400085E0EADC74DFCFBFCF9108958093C304A8
:1025500008958091C3040895E6ECF5E280879187A1
:102560006287738708951F93CF93DF93162FEA0135
:1025700004DDFC018181807CD1F5612F63706130C5
:1025800019F020F080E803C080EC01C080E4C0387E
:10259000D105E1F050F4C032D105A1F0C034D1052D
:1025A00099F06097C9F491E018C0C11592E0D9077D
:1025B00079F0CF3F93E0D90769F0C115D14061F4BC
:1025C00095E00BC092E009C093E007C094E005C01D
:1025D00096E003C097E001C090E0118226E02083DE
:1025E000982B918381818062818381E001C080E0AA
:1025F000DF91CF911F910895C0DCFC01818182FBA6
:10260000882780F90895CF93C82FB7DCFC0181811A
:1026100082FF0FC081818B7F81838C2F10DDFC01B5
:10262000908190FF06C09E7F90830780F085E02D0B
:10263000099581E0CF910895AF92BF92CF92DF923A
:10264000EF92FF920F931F93CF93DF93D82EC62E56
:102650005A017901F4DCEC018D2D8FDC9C01DC0149
:1026600011968C911197807C09F454C011968C912D
:102670001197807C803C21F011968C9182FD4AC09C
:102680009FB7F894888180FF02C09FBF43C08160DC
:1026900088839FBFA982BA82EB82FC821D821E8240
:1026A0000F83188791E0C11004C0E114F10409F010
:1026B00090E0888190FB81F98B7F8883D7FE02C0F0
:1026C000F90122C0D90111968C911197807C803C30
:1026D000C1F41196EC91E770E150E73040F4F0E07E
:1026E000EE0FFF1FE455FF4D6081718102C068E06D
:1026F00070E0C701EED1892B21F088818E7F88831D
:1027000009C0F90112821382168217828D2DB1DC65
:1027100081E001C080E0DF91CF911F910F91FF9088
:10272000EF90DF90CF90BF90AF900895EF92FF921F
:102730000F93CF93C82F21DC7C018C2F80DCDC0130
:10274000F70102E005939C9190FF1BC09E7F9C9334
:102750001796ED91FC911897309799F0D701C7FF24
:1027600005C016966D917C91179704C012966D91D5
:102770007C9113974C2F81E0CF910F91FF90EF90B8
:102780000994CF910F91FF90EF900895CF93C82FA8
:10279000CDDF8C2FF2DBFC011182CF9108950F93D6
:1027A000CF93C82FEADBFC0181818460818301E043
:1027B00006938C2FBBDF81E0CF910F9108951F927C
:1027C0000F920FB60F9211240F932F933F934F93B5
:1027D0005F936F937F938F939F93AF93BF93CF93A9
:1027E000EF93FF938091CB0487FF08C080E880932C
:1027F000CA040E94750B0E94210486C08091CB04FC
:1028000082FF18C084E08093CA0480912C2386FF45
:102810007BC08091CC0481FD77C099DD811174C0AB
:1028200080910723813011F4F4DB6EC0843009F00D
:102830006BC021C08091CB0481FF26C082E08093D1
:10284000CA048091242386FF5FC08091CC0481FD5F
:102850005BC07DDD811158C080910723823041F437
:1028600084E080930723E4E2F3E202E006934CC0A5
:10287000833009F049C0EDE2F3E204E00593E5E2BC
:10288000F3E204E0059340C08091CB0484FF25C0AF
:1028900080E18093CA04C1E08C2F48DF8C2F8068D0
:1028A00045DFCF5FC630C1F70E94580B1092C304BA
:1028B00010922523C093242383E480932523109230
:1028C0002D23C0932C2380932D2383EC92E28093BD
:1028D00028239093292368DB17C08091CB0486FFBF
:1028E00008C080E48093CA0480E034DB0E941F04A7
:1028F0000BC08091CB0485FF07C080E28093CA049F
:1029000081E028DB0E942004FF91EF91CF91BF91DD
:10291000AF919F918F917F916F915F914F913F9177
:102920002F910F910F900FBE0F901F9018951F922F
:102930000F920FB60F9211240F931F932F933F9373
:102940004F935F936F937F938F939F93AF93BF93B7
:10295000CF93DF93EF93FF938091CC0481FF1AC054
:1029600082E08093CC048091C5048195880FE4E2D5
:10297000F3E2E81BF109208131812452334283E0E4
:10298000369527958A95E1F7822F869520FD06C01A
:10299000C0E005C0DCDC882319F386C0C0E8C80F9E
:1029A0008C2FEBDAFC01208125FF7EC000E206932C
:1029B000C11174C080910723843019F438DBF4DA34
:1029C00073C000912623109127238091D0259091E8
:1029D000D125C0910323D091042398012C0F3D1FD2
:1029E0008217930718F48C010C1B1D0B8091CE25C8
:1029F0009091CF25A80163EC72E28C0F9D1F96D0B9
:102A0000C00FD11FC0930323D093042300341105BA
:102A100069F480910523909106238C0F9D1F2091CE
:102A2000CC253091CD258217930788F0C093D0250F
:102A3000D093D125E091D425F091D525309729F078
:102A40000995811102C0D7DA2FC0E3DA2DC0809139
:102A5000D0259091D125C817D907D9F4E091D42574
:102A6000F091D525309779F30995882361F320916A
:102A70000523309106238091032390910423820F34
:102A8000931F8093052390930623109203231092A3
:102A90000423E4E2F3E202E0069306C0C03811F436
:102AA000E8DB02C08C2FE5DAFF91EF91DF91CF9147
:102AB000BF91AF919F918F917F916F915F914F9156
:102AC0003F912F911F910F910F900FBE0F901F906C
:102AD0001895AA1BBB1B51E107C0AA1FBB1FA61755
:102AE000B70710F0A61BB70B881F991F5A95A9F7B7
:102AF00080959095BC01CD01089597FB072E16F4A3
:102B0000009406D077FD08D0E4DF07FC05D03EF442
:102B1000909581959F4F0895709561957F4F089589
:102B2000EE0FFF1F0590F491E02D0994FB01DC01ED
:102B300002C001900D9241505040D8F70895FB011A
:102B4000DC0101900D920020E1F70895F894FFCF89
:102B500040000CE02E0AFFFFFFFF5580008000615F
:102B60000A5B0A6B0A580A000064201F2000002834
:102B70002023200F2000000009023C0001010080FA
:102B8000FA0904000006FFFFFF000705810180002D
:102B9000010705820180000107058301800001070C
:102BA0000584018000010705850180000107058675
:102BB000018000011201000200000040EB0394BA02
:102BC00000020102000100000003000000000000FC
:102BD000000000000000000000004C6162726164AF
:102BE0006F72004573706F54656B00000403090435
:102BF0006465627567313233000106001000200001
:0A2C00004000800000010002FF0305
:00000001FF
